:100000000C9417060C9475290C94A2290C943F06A5
:100010000C943F060C943F060C943F060C943F064C
:100020000C943F060C943F060C94C50C0C943F06B0
:100030000C943F060C943F060C943F060C943F062C
:100040000C94CF290C943F060C94892D0C94C42D4C
:100050000C943F060C943F060C943F060C943F060C
:100060000C943F060C943F069F1CA61CA61C9F1CCC
:10007000A61CA61CA61CA61CA61CA61CA61CA61C70
:10008000A61CA61CA61CA61CA61C141CA61CA61CF2
:10009000A61CA61CA61C7E1BA61CA61CA61CA61C79
:1000A000A61CA61CA61CA61CA61CA61CA61CA61C40
:1000B000A61CA61CA61C201C201C201C201C201CCE
:1000C000201C201C201C201CA61CA61CA61CA61C38
:1000D000A61CA61C7E1B1F1C1F1C1F1C1F1CA61C55
:1000E000301C381C401C481C501C581C601C681CD0
:1000F000721C7C1C861C901CC31B831BA61CA61C8C
:10010000A61CA61C141CA61CA61CA61CA61CA61C71
:10011000A61CA61CA61C1E1C1E1C1E1C1E1CA61CEF
:10012000301C381C401C481C501C581C601C681C8F
:10013000721C7C1C861C901CC31B831BA61CA61C4B
:10014000A61CA61C141CD71CD71CD71CD71CD71C3C
:10015000D71CD71CD71CD71CD71CD71CD71CD71C07
:10016000F71DF71DF71DF71DF71DF71D1E1D281D97
:10017000321D3C1DA21DAC1DBA1DCB1D681ED81E14
:10018000A91EAE1EB31EB81EBD1EC21EC71ED81E9F
:10019000D21EF125062612261B2628264E26562676
:1001A00079266626456E746572206D656E752E2EF5
:1001B0002E00546F67676C6564206D6963726F50C1
:1001C000504D00546F67676C656420696E76657288
:1001D0007465642050504D2100546F67676C6564EE
:1001E000205458206D7574696E672100546F6767DD
:1001F0006C65642074656C656D657472792100505E
:10020000726F746F636F6C206572726F72207769A2
:1002100074682052580054696D656F757420776852
:10022000656E20636F6E6E656374696E6720746FB0
:1002300020525800507265737320616E79206B658F
:100240007920746F2063616E63656C00436F6E6E1E
:10025000656374696E6720746F2052582C20706F2C
:100260007765722075702074686520525820287751
:100270006974682062696E6420706C7567206966B5
:10028000206E6F74207573696E6720616C77617979
:10029000732062696E642900546F67676C6564201F
:1002A00027696D6D656469617465206F757470751B
:1002B000742700546F67676C65642027736C6176E0
:1002C00065206D6F64652700546F67676C656420F7
:1002D00027616C776179732062696E642700546FBF
:1002E00067676C65642050504D206368616E6E6571
:1002F0006C206C696D6974005365742052535349C6
:1003000020696E6A656374696F6E206368616E6EE2
:10031000656C2028303D3D64697361626C6529001D
:100320005365742050504D206D696E696D756D2058
:1003300073796E630053657420626561636F6E202C
:10034000696E74657276616C0053657420626561D4
:10035000636F6E2064656C6179005365742062651B
:1003600061636F6E206672657175656E6379206971
:100370006E20487A3A20303D64697361626C652C66
:100380002050783D504D52206368616E6E656C2040
:10039000782C2046783D465253206368616E6E6526
:1003A0006C2078005365742050574D2073746F7023
:1003B0002064656C61792028302064697361626C07
:1003C00065642C20312D323535203D3D20302E31D5
:1003D00073202D2035306D696E29005365742050CF
:1003E000504D2073746F702064656C6179202830E3
:1003F0002064697361626C65642C20312D3235355F
:10040000203D3D20302E3173202D2035306D696E1A
:100410002900536574206661696C736166652064A8
:10042000656C61792028302064697361626C656451
:100430002C20312D323535203D3D20302E3173209A
:100440002D2035306D696E29002A2A2A2A2A2A2A67
:100450002A2A2A2A2A2A2A2A2A2A2A2A2A2A2A2AFC
:100460002A2A2A2A2A2A0052582041636B656420CE
:100470002D2072657665727420737563636573737E
:1004800066756C21002A2A2A2A2A2A2A2A2A2A2A36
:100490002A2A2A2A2A2A2A2A2A2A2A2A2A2A2A2ABC
:1004A0002A2A002A2A2A2A2A2A2A2A2A2A2A2A2AD6
:1004B0002A2A2A2A2A2A2A2A2A2A2A2A2A2A2A2A9C
:1004C0000052582041636B6564202D207570646173
:1004D0007465207375636365737366756C21002A98
:1004E0002A2A2A2A2A2A2A2A2A2A2A2A2A2A2A2A6C
:1004F0002A2A2A2A2A2A2A2A2A2A2A2A0056616CE1
:1005000069642063686F69636573206172653A206E
:100510005B315D2D5B31365D20286368616E6E65F1
:100520006C20312D31362900536574206F7574703D
:10053000757420666F7220706F727420005B585D56
:100540002061626F7274206368616E6765732061F9
:100550006E64206578697420525820636F6E6669F6
:1005600067005B535D207361766520736574746901
:100570006E677320746F205258005B525D20726565
:10058000766572742052582073657474696E67734F
:1005900020746F2064656661756C747300557365B3
:1005A000206E756D62657273205B312D445D207421
:1005B0006F206564697420706F727473205B452DC1
:1005C000515D20666F722073657474696E67730085
:1005D000202D20726563656976657220636F6E6693
:1005E0006967757261746F722C207278207377203E
:1005F000000A0A6F70656E4C52536E672000536597
:10060000742073657269616C2062617564726174D3
:10061000653A200056616C69642063686F696365A0
:10062000733A2031202D20342B34202F2032202DDE
:100630002038202F2033202D20382B34202F203419
:10064000202D203132202F2035202D2031322B3407
:10065000202F2036202D203136005365742043682A
:10066000616E6E656C20636F6E6669673A20005339
:1006700065742044617461726174652028302D3284
:10068000293A200053657420486F70206368616EBA
:100690006E656C7320286D61782032342C20736570
:1006A0007061726174656420627920636F6D6D6141
:1006B00073292076616C69642076616C756573209E
:1006C000312D3235353A2000536574206368616EF0
:1006D0006E656C2073706163696E672028783130B5
:1006E0006B487A293A200053657420524620706F77
:1006F0007765722028302D37293A20005365742001
:100700005246206D616769632028686578292065F5
:100710002E672E20307844454144463030443A20FC
:10072000005365742062617365206672657175653A
:100730006E63792028696E20487A293A20005B5A36
:100740005D20656E74657220726563656976657299
:1007500020636F6E66696775726174696F6E20756C
:1007600074696C79005B465D20646973706C6179B3
:100770002061637475616C206672657175656E6366
:100780006965732075736564005B525D2063616CFD
:1007900063756C6174652072616E646F6D206B654A
:1007A0007920616E6420686F70206C697374005BDF
:1007B000495D207265696E697469616C697A65204A
:1007C00073657474696E677320746F20736B6574DE
:1007D00063682064656661756C7473005B585D20A6
:1007E000726576657274206368616E6765732061F7
:1007F0006E642065786974206D656E75005B535D6D
:1008000020736176652073657474696E67732074F4
:100810006F20454550524F4D20616E6420657869C8
:1008200074206D656E7500557365206E756D62651B
:100830007273205B302D395D20746F20656469749C
:1008400020706172616D657465727300202D205394
:10085000797374656D20636F6E6669677572617414
:10086000696F6E000A0A6F70656E4C52536E672096
:10087000005129204F7574707574206265666F721F
:1008800065206C696E6B20283D465329203A200074
:10089000502920536C617665206D6F646520286552
:1008A00078706572696D656E74616C293A20004FCD
:1008B000292054696D65642042494E4420617420AA
:1008C0007374617274757020203A20004E29205094
:1008D000504D206F7574707574206C696D69746506
:1008E0006420202020203A200044495341424C45B6
:1008F00044004D292050504D205253534920746FCD
:10090000206368616E6E656C202020203A20004CC8
:10091000292050504D206D696E696D756D20737979
:100920006E63202875732920203A200044495341E2
:10093000424C4544004B29204661696C73616665F1
:1009400020626561636F6E20696E74762E20283197
:100950002D32353573293A20004A29204661696CC9
:100960007361666520626561636F6E2064656C61AA
:10097000792028302D323535203D3E20313073200E
:100980002D203135306D696E293A200049292046E5
:1009900061696C7361666520626561636F6E206674
:1009A00072712E203A200048292050574D20737430
:1009B0006F702064656C6179202020202020203A0F
:1009C000200047292050504D2073746F70206465BB
:1009D0006C6179202020202020203A200046292008
:1009E0004661696C736166652064656C617920207D
:1009F00020202020203A200050574D206368616E4F
:100A00006E656C200066756E6374696F6E3A2000C7
:100A10002920706F72742000506F776572546F7761
:100A2000657200445446205548462033322D626991
:100A3000742031306368004F70656E4C52536E679E
:100A40005258206D696E6920342F36636800466CF9
:100A50007974726F6E2F4F72616E676552582055B0
:100A600048462038636800525820747970653A20EF
:100A70000044697361626C656400487A00203D3D02
:100A8000200043616C63756C617465642070616300
:100A90006B657420696E74657276616C3A200042F1
:100AA00029204D6963726F202868616C6629205087
:100AB000504D202020203A00412920496E76657251
:100AC0007465642050504D20696E20202020203A0B
:100AD000003029204D7574652062757A7A65722020
:100AE000286D6F73746C79293A0039292053657227
:100AF00069616C2062617564726174653A00736D3E
:100B0000617274506F7274004672536B7900547244
:100B1000616E73706172656E740044697361626CBA
:100B200065640038292054656C656D657472793A86
:100B300020202020202020003729204368616E6E6D
:100B4000656C20636F6E6669673A20200036292045
:100B500044617461726174652028302D32293A2015
:100B6000202000352920486F70206368616E6E6513
:100B70006C733A2020202020003429204368616EC5
:100B80006E656C2073706163696E673A2020003374
:100B90002920524620706F7765722028302D372922
:100BA0003A202020003229205246206D6167696377
:100BB0003A202020202020202020003129204261BE
:100BC0007365206672657175656E63793A202020C1
:100BD0000000000000240027002A0000000000257B
:100BE0000028002B0000000000230026002900043C
:100BF00004040404040404020202020202030303C4
:100C000003030301020408102040800102040810BD
:100C1000200102040810200000000700020100006B
:100C20000304060000000000000000006C2F1124E7
:100C30001FBECFEFD8E0DEBFCDBF13E0A0E0B1E034
:100C4000EAE1F1E602C005900D92A839B107D9F7A3
:100C500016E0A8E9B3E001C01D92AD35B107E1F798
:100C60001CE0CEE2DCE004C02297FE010E94683066
:100C7000CC32D107C9F70E94B12F0C948B300C9461
:100C80000000A0E0B0E0E7E4F6E00C943730EC01BF
:100C9000A880B980CA80DB80A114B104C104D1044A
:100CA00041F484E2A82E89EDB82E8BE5C82E87E0AA
:100CB000D82EC601B5012DE133EF41E050E00E948E
:100CC000143027EA31E440E050E00E94C02F7B015D
:100CD0008C01C601B5012DE133EF41E050E00E94E7
:100CE0001430CA01B9012CEE34EF4FEF5FEF0E94D0
:100CF000C02F6E0D7F1D801F911F97FF04C0615094
:100D0000704080409048688379838A839B839B01ED
:100D1000AC015F77B901CA01CDB7DEB7EAE00C9448
:100D200053300E944106089581EB92E00E944106F3
:100D300008956093B1027093B2028093B3029093CE
:100D4000B4020895A0E0B0E0E8EAF6E00C94303098
:100D5000EC012B016A016115710519F0FB0191830A
:100D60008083C114D10449F0C6010297839728F00B
:100D700020E030E040E050E0DCC0A9908A2D90E017
:100D80000E948030892BC9F7FDE2AF1621F4A990AB
:100D90003324339405C08BE2A81609F4A9903324B8
:100DA000C114D10421F0E0E1CE16D10411F5F0E335
:100DB000AF1669F48881883711F0883541F4A9802D
:100DC000229682E0382A20E1C22ED12C12C0C11412
:100DD000D10479F4E0E3AE1659F199E9E92E99E9E5
:100DE000F92E99E9092F99E1192F8AE0C82ED12C03
:100DF0003AC0FAE0CF16D10491F080E1C816D104D0
:100E000029F0E8E0CE16D104F9F415C0BFEFEB2EBF
:100E1000BFEFFB2EBFEF0B2FBFE01B2F24C0A9E9B4
:100E2000EA2EA9E9FA2EA9E90A2FA9E11A2F1BC077
:100E3000F8E0CF2ED12CEFEFEE2EEFEFFE2EEFEFFE
:100E40000E2FEFE11E2F0FC09601442737FD40956E
:100E5000542F6FEF7FEF8FEF9FEF0E94F22FC901AA
:100E6000DA017C018D0120E030E040E050E060E0FC
:100E70003601882477FC8094982C70EDB72EBA0C3C
:100E8000F9E0FB1570F48A2D81548A3118F499EC3D
:100E9000B92E06C08A2D81568A3148F589EAB82EC6
:100EA000BA0C8B2D90E08C159D050CF56F3FE9F089
:100EB000E216F30604071507B8F0CA01B901A40148
:100EC00093010E94C02F9B01AC018B2D90E0A0E00C
:100ED000B0E0280F391F4A1F5B1F281739074A0740
:100EE0005B0710F061E001C06FEFA990C6CF41141D
:100EF000510451F0662311F0219703C031FE04C064
:100F00002297F201D183C08330FE07C050954095EF
:100F1000309521953F4F4F4F5F4F67FF0AC082E2E8
:100F200090E090935C0680935B062FEF3FEF4FEFCE
:100F30005FEFB901CA01CDB7DEB7E1E10C944C30E7
:100F4000FC0188279927E89421912032E9F3293080
:100F500010F02E30C8F32B3241F02D3239F4689462
:100F600004C00E94F507820F911D219120532A3061
:100F7000C0F31EF4909581959F4F089548E953E082
:100F80000E94C3070895009731F4DA018D919C9176
:100F9000009709F40EC0DC01FB013D912191222351
:100FA00019F03217C9F3FACF332331F4DA011D9265
:100FB0001C928827992708951197AF93BF93FB013F
:100FC0003D912191321771F4332321F48827992719
:100FD000119702C01E921196FA01A193B0839F91BE
:100FE0008F910895222369F7EACF7AE0979F902D99
:100FF000879F802D910D1124089580919A0381304F
:1010000019F482E080939A0380919A03833019F453
:1010100084E080939A030895E3E0F0E089E0809310
:101020005700849190E08670863009F491E0892F12
:1010300008951F93182F0E940C08882379F09FB7FA
:1010400081E08093A305F894A89588E180936000DF
:1010500010936000112309F0A8959FBF1F91089578
:10106000382F20E08091350590913605822793270F
:1010700040E061E270E19C01220F331F97FF04C042
:10108000C9018627972701C0C9014F5F483099F7EA
:101090009093360580933505089587E38093D003B8
:1010A00080E092ECA1E0B0E08093D1039093D20372
:1010B000A093D303B093D40387E08093DD0380E053
:1010C00091EAACEBB3E38093D5039093D603A0935E
:1010D000D703B093D80385E08093DE038DEE9EEFB7
:1010E000ADEABEED8093D9039093DA03A093DB03BE
:1010F000B093DC03AFEDB3E080E090E0863010F019
:10110000E0E004C0FC01EF57FC4FE081ED93019655
:101110008831910599F782E08093F7038AE0809304
:10112000F803089580E09EECADEEB4E380939D0358
:1011300090939E03A0939F03B093A00380E090E060
:10114000A0E0B0E58093A1039093A203A093A30332
:10115000B093A403E5EAF3E080E081938F5F8031F0
:10116000E1F708958436910520F4BC0180E090E019
:1011700025C08E3B910550F48A559040BC0180E01B
:1011800090E02AE030E040E050E016C0823D91055A
:1011900050F4845B9040BC0180E090E024E630E0B5
:1011A00040E050E009C08D5C9040BC0180E090E0E0
:1011B00028E532E040E050E00E94C02F24E630E015
:1011C00040E050E00E94C02F089590E08C599F4F5E
:1011D0000E94B2080895DC019896EC91F0E0E77067
:1011E000F070E758FC4F808108958F929F92AF92E4
:1011F000BF92CF92DF92EF92FF920F931F938C01D9
:101200000E94EB08D80197962C9130E043E150E022
:10121000249FF001259FF00D349FF00D1124EB5415
:10122000FD4F80809180A280B38090E00F96AA2726
:1012300097FDA095BA2FBC01CD0120E43FE14DE719
:1012400050E00E94C02FA50194010E94F22F690175
:101250007A0180ED97E0A0E0B0E0C80ED91EEA1E4A
:10126000FB1ED80198968C91887181F060E07EEE2B
:101270008AEB9BE0A50194010E94F22F28513C4F7C
:101280004F4F5F4FC20ED31EE41EF51E87EE93E054
:10129000A0E0B0E0C80ED91EEA1EFB1EC701B601D1
:1012A00028EE33E040E050E00E94F22FCA01B9017D
:1012B00028EE33E040E050E00E94C02F1F910F91D4
:1012C000FF90EF90DF90CF90BF90AF909F908F9066
:1012D00008958F3F910509F010F480E0089522E011
:1012E0008030920710F481E008958050934010F010
:1012F00083E0089582E00895CF92DF92FF920F93EA
:101300001F93CF93DF93F82FEB016A01182F1695E7
:10131000E0E088819981D6018C938A819B81119626
:101320008C9311978C819D8112968C9312978E814C
:101330009F8113968C931397288139814A815B8111
:101340006C817D818E819F819295990F990F907C00
:10135000832F8370982B852F8370880F880F982B8D
:10136000872F83708295807F982B14969C9385E0BD
:1013700090E0C80ED91E2896EF5F1E1750F6F0FFBA
:1013800021C0888199810E946909F82E8A819B81F8
:101390000E946909182F8C819D810E946909082F7C
:1013A0008E819F810E946909F294FF0CFF0C70EC02
:1013B000F7221295107F1F29182B000F000F012B09
:1013C000D6010C93DF91CF911F910F91FF90DF9089
:1013D000CF90089523E08032920718F420E030E0A7
:1013E00026C023E0883E920748F49C012F513340E9
:1013F00054E0369527955A95E1F719C027E0803DCE
:10140000920720F49C012C5D334011C028E08839FC
:10141000920718F02FEF33E00AC09C01285C374098
:1014200044E0369527954A95E1F72D503C4FC90188
:1014300008958C30910548F49C0174E0220F331F0D
:101440007A95E1F7285D3C4F17C023E0843F92076F
:1014500020F49C0124523C4F0FC024E080309207BE
:1014600018F020E938E008C09C012657334F64E0AB
:10147000220F331F6A95E1F7C90108959C01369543
:10148000279525753575821B930B9C0136952795FD
:10149000369527952373337383739373280F391FFE
:1014A000C901E4E096958795EA95E1F7820F931FCD
:1014B0008F709F7021E031E0AC01429FC001439FDB
:1014C000900D529F900D1124892F0895882339F093
:1014D0002D9800002B9A00002D9A000008952D9859
:1014E00000002B9800002D9A000008952D9A00000E
:1014F00083B12D98000090E0B4E096958795BA9559
:10150000E1F7817008950F931F93082F5C9A2D982F
:101510005C9810E0802F80780E94660A000F1F5FA1
:101520001830C1F72D981F910F9108958F770E9461
:10153000830A08950F931F93082F10E0802F80785F
:101540000E94660A000F1F5F1830C1F72D981F9187
:101550000F9108950F931F932D9880E000E0182FAE
:10156000110F0E94760A810F0F5F0830C1F71F919B
:101570000F9108950E94960A0E94AA0A5C9A089503
:101580001F93162F80680E94830A812F0E949A0A57
:101590005C9A1F9108951F931091D9031827E0EDCD
:1015A000F3E0E80FF11D89E767850E94C00A8DE32B
:1015B000612F0E94C00A82E4612F0E94C00A1F911D
:1015C000089586E20E94BA0A08950F931F938C0132
:1015D0008CE1F80164810E94C00A8DE1F801658107
:1015E0000E94C00A8EE1F80166810E94C00A80E272
:1015F000F80167810E94C00A81E2F80160850E94BB
:10160000C00A82E2F80161850E94C00A83E2F80103
:1016100062850E94C00A84E2F80163850E94C00AC4
:1016200085E2F80164850E94C00A8AE2F8016585B6
:101630000E94C00A8EE6F80166850E94C00A8FE605
:10164000F80167850E94C00A80E7F80160890E945E
:10165000C00A81E7F80161890E94C00A82E7F801A7
:1016600062890E94C00A1F910F910895EF92FF9224
:101670000F931F93CF93DF937B018C01603028E39E
:1016800072072CE982072CE1920728F520E836E959
:1016900048E950E00E94F22FE9016897B90180E023
:1016A00090E020E839E647E65FEF0E94C02F6E0D1C
:1016B0007F1D801F911F32E0660F771F881F991FC3
:1016C0003A95D1F721E732E040E050E00E94F22F56
:1016D000890180E421C020E03DE241E351E00E9425
:1016E000F22FE9016897B90180E090E020E033ED46
:1016F0004EEC5EEF0E94C02F6E0D7F1D801F911F6C
:10170000660F771F881F991F21E732E040E050E005
:101710000E94F22F890180E69E012F71622F680FCF
:1017200085E70E94C00A86E7612F0E94C00A87E70A
:10173000602F0E94C00ACDB7DEB7E6E00C945730A8
:10174000682F8DE60E94C00A08959F92AF92BF92C3
:10175000CF92DF920F93DF93CF9300D000D0CDB71D
:10176000DEB7982E83E00E94BA0A8093F90384E0E2
:101770000E94BA0A8093FA0386E060E00E94C00AE1
:1017800087E061E00E94C00A89E06FE70E94C00A1A
:101790008AE065E00E94C00A8BE062E10E94C00A14
:1017A0008CE065E10E94C00A8DE06DEF0E94C00AE6
:1017B0008EE060E00E94C00A992019F084E193E075
:1017C00008C08091F70323E1829FC00111248B544C
:1017D0009D4F0E94E50A80E36CE80E94C00A82E304
:1017E0006FE00E94C00A83E362E40E94C00A84E3BF
:1017F0006AE00E94C00A85E36AE20E94C00A86E3AA
:101800006DE20E94C00A87E364ED0E94C00A88E38B
:1018100060E00E94C00A89E360E00E94C00A99204B
:1018200049F065E8A62E61ECB62E61ECC62E6EED91
:10183000D62E08C0A090D903B090DA03C090DB0385
:10184000D090DC030AE38D2D9927AA27BB27898333
:101850009A83AB83BC83802F69810E94C00A802F4A
:101860008B5F69810E94C00ADC2CCB2CBA2CAA2485
:101870000F5F0E3341F783E46FEF0E94C00A84E4E8
:101880006FEF0E94C00A85E46FEF0E94C00A86E4F1
:101890006FEF0E94C00A992019F08DE666E003C040
:1018A0008DE66091DD030E94C00A89E760E00E9436
:1018B000C00A8AE76091DE030E94C00A83E760E005
:1018C0000E94C00A84E760E00E94C00A992029F0C3
:1018D00060E071EA8CEB93E308C06091D5037091EE
:1018E000D6038091D7039091D8030E94360B0F90B6
:1018F0000F900F900F90CF91DF910F91DF90CF90CD
:10190000BF90AF909F90089587E061E00E94C00A69
:101910008EE764E20E94C00A88E063E00E94C00A89
:1019200088E060E00E94C00A87E065E00E94C00A8B
:1019300085E062E00E94C00A83E00E94BA0A8093B8
:10194000F90384E00E94BA0A8093FA030895582F9D
:1019500040919E04842F90E0FC01EF70F0709F0195
:101960002F5F3F4F74E0959587957A95E1F728179B
:10197000390751F0E257FB4F5083842F8F5F8F70F0
:10198000407F842B80939E0408951F920F920FB680
:101990000F9211241F932F933F934F935F936F9355
:1019A0007F938F939F93AF93BF93CF93DF93EF93E7
:1019B000FF93C0918600D09187002091E20430917E
:1019C000E3048091C104882309F062C0BE01621B58
:1019D000730B2091A1033091A2034091A303509176
:1019E000A40325FD02C07695679589E0653C7807DC
:1019F000B8F1809147031CE1569547953795279597
:101A00001A95D1F7211531054105510521F421E041
:101A100030E040E050E090E0A0E0B0E02817390767
:101A20004A075B07D0F4809147038F3FB1F020E075
:101A30000EC0E22FF0E0EE0FFF1FDF01AE53BB4FF1
:101A40008D919C91E95DFC4F918380832F5F809104
:101A50004703281770F31092C0041092470318C070
:101A600082E06D3B780760F180914703803140F55B
:101A700010914703CB010E94EA09E12FF0E0EE0F3D
:101A8000FF1FEE53FB4F918380831F5F109347032B
:101A9000D093E304C093E204FF91EF91DF91CF91E3
:101AA000BF91AF919F918F917F916F915F914F9176
:101AB0003F912F911F910F900FBE0F901F9018957F
:101AC0008FEF80934703E4CF83E0809380008AE91F
:101AD000809381008091A10386FD05C080918100E3
:101AE0008064809381008FEF9FEF909389008093B3
:101AF000880080916F00806280936F0008956F303E
:101B000018F086958058089589E0689F802D1124EB
:101B10000895882319F460E071E002C063E071E089
:101B200089E396E00E94742D0895A0E0B0E0EBE90F
:101B3000FDE00C943930182F0E94252A9B01AC013E
:101B400080912F0590913005A0913105B09132051B
:101B500069017A01C81AD90AEA0AFB0AD701C60143
:101B600089589341A040B04010F010922E05209368
:101B70002F05309330054093310550933205209165
:101B8000C104822F81508230E8F580912E05882390
:101B900009F44FC1813011F482E0BCC1803108F0FA
:101BA00035C1E82FF0E0EE53FB4F10838F5F809339
:101BB0002E05803109F0B0C1A4ECB4E0213039F435
:101BC0001196EC911197E695E6958C9109C08D914F
:101BD0009C911197E92FE695E695E6959695879560
:101BE000E03140F4F0E090E0EE0FFF1FE95DFC4FC4
:101BF000918380831092C004129684E0A23DB807BE
:101C0000E9F68AC1233009F004C180912E058823AA
:101C100021F41F3009F080C10CC1883130F4E82F65
:101C2000F0E0EF53FB4F108374C1883109F0EEC030
:101C3000112309F0EBC0C0E0D0E00BE010E0DE01C2
:101C400063E0AA0FBB1F6A95E1F7C09FB001C19F77
:101C5000700DD09F700D1124FB01EE53FB4F80815E
:101C60002181922F977095958795FD01EE0FFF1FAB
:101C7000E95DFC4F91838083FB01ED53FB4F308185
:101C80003695369536952181422F4295440F407EF8
:101C9000842F832B269526952695922F97709595C0
:101CA0008795FD01EE0FFF1FE75DFC4F9183808359
:101CB000FB01EC53FB4F808182958695869583705E
:101CC0004181942F990F990F292F282B42954695E2
:101CD0004695437082818170880F880F382F342B8E
:101CE00035952795FD01EE0FFF1FE55DFC4F318314
:101CF0002083FB01EA53FB4F308136952181422F2F
:101D0000479544274795842F832B2695922F9770CC
:101D100095958795FD01EE0FFF1FE35DFC4F9183C5
:101D20008083FB01E953FB4F308132953F70218165
:101D3000422F4295407F842F832B22952F70922F24
:101D4000977095958795FD01EE0FFF1FE15DFC4FA4
:101D500091838083FB01E853FB4F8081881F882794
:101D6000881F4181942F990F292F282B441F442726
:101D7000441F82818370880F382F342B3595279527
:101D8000FD01EE0FFF1FEF5CFC4F31832083FB0151
:101D9000E653FB4F3081369536952181422F42958F
:101DA000440F440F407C842F832B26952695922F39
:101DB000977095958795AA0FBB1FFD01ED5CFC4FB1
:101DC0009183808365537B4FFB012081229526956B
:101DD00027704181342F330F330F330F832F822B22
:101DE000942F92959695977095958795AB5CBC4F7F
:101DF00011969C938E932196C230D10509F01FCF86
:101E00008091D80483FD02C01092C00410922E0568
:101E100083C0243009F080C040912E05442359F43A
:101E2000183AB1F4109236051092350588EA0E94EE
:101E3000300881E06FC0413019F41093330504C0BD
:101E4000423031F410933405812F0E9430085DC078
:101E500060913405262F30E0220F331FE42FF0E08D
:101E6000C90102968E179F0734F0433268F7E15498
:101E7000FB4F1083E9CF2D5F3F4F409135055091C7
:101E80003605E217F30749F4912F80E048275927D8
:101E9000509336054093350538C0812F90E04817A0
:101EA000590789F580913305813069F5613118F062
:101EB00080E180933405D090340542ECE42E44E078
:101EC000F42E00E010E01BC0F701D081C0E081815A
:101ED00090E08C2B9D2B33E0969587953A95E1F712
:101EE0000E94EA09F801EE0FFF1FE95DFC4F9183A4
:101EF00080830F5F1F4F82E090E0E80EF91E0D1502
:101F000018F31092C00410922E0580912E0588239C
:101F100019F08F5F80932E05CDB7DEB7E8E00C9403
:101F20005530FF920F931F93CF93DF93182F092FF4
:101F3000F62E8EE30E94C00A212F302FC901EC013A
:101F400010E005C08FE769910E94C00A1F5F1F154E
:101F5000C8F385E064E00E94C00A83E00E94BA0AE8
:101F60008093F90384E00E94BA0A8093FA030E94E6
:101F7000252A6093FB037093FC038093FD039093E9
:101F8000FE0387E069E00E94C00A81E080939A0323
:101F9000CDB7DEB7E5E00C9458300E94910F8091E8
:101FA0009A038130D9F40E94252A2091FB033091B5
:101FB000FC034091FD035091FE03621B730B840BE5
:101FC000950B605A76488140904040F4E8CF89E311
:101FD00096E067E071E00E94742D089580919A0365
:101FE0008130A9F3089589E396E06EE70E942C2FD3
:101FF0000895A0E0B0E0EFEFFFE00C9438306C0102
:1020000089E396E06EE70E942C2F760100E010E055
:10201000C0E0D0E0B0E2BB2E0AC00830110521F4C8
:102020009E012095F60120870894E11CF11CF70120
:102030006081862F8D57823040F489E396E06DE70A
:102040000E942C2FF70160816B2589E396E00E94A6
:102050002C2F0115110551F0F70180819E01280FE9
:10206000311DC32FDD27C20FD31FD0700F5F1F4F4D
:102070000930110591F6CDB7DEB7E9E00C94543084
:10208000A9E0B0E0E6E4F0E10C943F30382FE62F11
:102090008091A30490E0019664E270E00E94DF2F3B
:1020A000982F8093A30488E9898380E18A83913003
:1020B00071F0913028F0923099F09330E1F416C02D
:1020C00085E08B8381EF8C832F5F2D8317C09B83EB
:1020D00081EF8C8384E6489FC00111249D830EC04C
:1020E00084E08B8381EF8C833D8308C09B8381EFE9
:1020F0008C83ED8303C00E94F30F04C0CE010196D0
:102100000E94F90F2996E2E00C945B300F931F9325
:10211000CF93DF93182F092F89E396E06EE70E9493
:102120002C2F212F302FC901EC0110E000E2888113
:102130008D57823040F489E396E06DE70E942C2FA2
:1021400088818027888389E396E069910E942C2FFB
:102150001F5F193061F789E396E06EE70E942C2F2C
:10216000DF91CF911F910F910895A9E0B0E0EBEBC3
:10217000F0E10C943F30382F8091A304882379F448
:102180008EEF89833A836B83842F90E095958795B2
:102190008C832D83198618861F821E822FC0409142
:1021A0009E04842F90E09C012F70307054E0959530
:1021B00087955A95E1F78217930721F18DEF89836F
:1021C0001A821B82DE01149620E008C0E257FB4F02
:1021D00080818D93405F2F5F263069F0842F90E0DF
:1021E000FC0134E0F595E7953A95E1F78F70907032
:1021F000E817F90759F740939E042A83CE01019608
:102200000E9486108091A30490E0019666E070E041
:102210000E94DF2F8093A3042996E2E00C945B30A8
:102220009F92AF92BF92CF92DF92EF92FF920F9365
:102230001F93B82EA62ED42EC22E902E0E94252A91
:102240007B018C0180918D0420919F043091A0042A
:102250004091A1045091A2048823B1F0D801C70194
:10226000821B930BA40BB50B815E9E42A040B04035
:1022700020F12C2DDC1408F42D2D8B2D6A2D422FEE
:10228000292D0E94401011C0D801C701821B930B59
:10229000A40BB50B81539547A040B04070F08B2D37
:1022A0006A2D4D2D2C2D0E94B510E0929F04F092C6
:1022B000A0040093A1041093A2041F910F91FF901A
:1022C000EF90DF90CF90BF90AF909F90089589E3FB
:1022D00096E0609100040E942C2F08951F93182F00
:1022E00089E396E0612F0E942C2F809100048127C2
:1022F000809300041F9108951F93192F0E946E115F
:10230000812F0E946E111F910895DF92EF92FF922C
:102310000F931F93D82E7B011092000409E316E05F
:10232000C80165EB0E942C2FC80162E60E942C2F89
:102330008D2D0E946E11C7010E947C111F910F917B
:10234000FF90EF90DF900895E82FF0E0E456FC4F07
:10235000E185E03158F4F894F0E0EE0FFF1FE95DFD
:10236000FC4F0190F081E02D78940DC0E03129F010
:10237000E13129F0E0E0F2E006C082E101C083E152
:102380000E94792BFC01CF0108958CE060E00E944F
:10239000AA2A8BE061E00E94AA2A8DE061E00E94F7
:1023A000AA2A82E060E00E94AA2A84E061E00E94FA
:1023B000AA2A0895EF92FF920F931F93009771F14D
:1023C0009C0140E050E068E478EE81E090E00E94FB
:1023D0001430C901DA017C018D0183E161E00E94C2
:1023E000162B8FEFE816F1040105110539F030F0D6
:1023F000FFEFEF2EF12C012D112D0AC0E114F10495
:102400000105110529F4E1E0EE2EF12C012D112D2D
:10241000E092B3008091B000806107C083E160E08A
:102420000E94162B8091B0008F7E8093B0001F9188
:102430000F91FF90EF900895A0E2B0E0E2E2F2E1A8
:102440000C9437308CE00E94BA0A882389F589E31E
:1024500096E063E171E00E94742D5E9A409A80E0FC
:102460000E94A50B0E94840C5E98409821C089E3CD
:1024700096E00E94F32E482F8091C104882321F01A
:10248000842F0E94950D14C080912C05E82FF0E058
:1024900031969F012F713070319780912B0590E01C
:1024A0002817390729F0EE5FFA4F408320932C0557
:1024B00089E396E00E94B92E892BC9F680919A0390
:1024C000843009F08EC00E94252A6093B004709376
:1024D000B1048093B2049093B30461157105810532
:1024E000910561F481E090E0A0E0B0E08093B00459
:1024F0009093B104A093B204B093B3048091BC0450
:102500009091BD0481609093BD048093BC0483E0EE
:1025100080939A038FE70E94960A09EF14E00E94C5
:10252000AA0AF80181938F01F5E002301F07B9F77D
:102530004091E4048091F904282F30E0842F90E04A
:102540008227932786FF40C080E448274093E40415
:10255000C90188739070C89709F510E014C01F5F17
:102560008091F803E12FF0E084FF06C0E750FB4FB5
:1025700080810E94A70C07C0E750FB4F89E396E0DB
:1025800060810E942C2F212F30E08091F90490E08F
:10259000877090708217930714F716C02F733070EE
:1025A000232B91F48091FA048093B4048091FB046E
:1025B0008093B6048091FC048093B7048091FF045B
:1025C0008093BE041092BF0480912D05813019F4D0
:1025D00082E080932D0580912D05833011F41092B7
:1025E0002D050E94252A5B016C018091B804909111
:1025F000B904A091BA04B091BB040097A105B1053C
:10260000C9F086017501E81AF90A0A0B1B0BD801FB
:10261000C701885B9B40A040B04060F00E94E10A87
:102620008093B5041092B8041092B9041092BA04C1
:102630001092BB0480ED93E00E94F5082091AC0459
:102640003091AD044091AE045091AF048601750104
:10265000E21AF30A040B150BE616F706080719072A
:1026600008F428C1A092AC04B092AD04C092AE04AC
:10267000D092AF04A8958091C0048830A0F08091DA
:10268000A1039091A203A091A303B091A4032CE114
:10269000B695A795979587952A95D1F70097A105A7
:1026A000B10509F0A7C18091C0048F5F8093C00479
:1026B000E090B004F090B1040091B2041091B30422
:1026C000E114F1040105110511F180ED93E00E9480
:1026D000F508AE18BF08C00AD10A6A157B058C053B
:1026E0009D0588F48091A10384FD04C080ED97E0EE
:1026F0000E94DA111092B0041092B1041092B20448
:102700001092B30404C080E090E00E94DA1190912E
:10271000E404907C9093E40400912C0510912B0527
:102720000117B1F180912D05823091F59058909369
:10273000E40480ED93E00E94EB08893010F048E05B
:1027400002C0482F415030E013C03F5FA32FB0E0DC
:10275000812F90E0FC01EE5FFA4F2081FD01EC51EA
:10276000FB4F2083AE5DBA4F2C930196182F1F713B
:10277000341710F4101749F710932B05832F895C39
:102780009091E404892B8093E404309322051AC0CD
:1027900020912D052430D1F490912205E3E2F5E05B
:1027A000A5EEB4E0292F30E02E0F3F1F02C081912B
:1027B0008D93E217F307D9F7995C8091E404982B85
:1027C0009093E40483E080932D0538C08091A704A2
:1027D000823061F491609093E4045E9A409A05EA35
:1027E00013E07E010894E11CF11C11C09093E404F5
:1027F0005E984098222319F481E080932D05809102
:102800002D05833061F784E080932D05E8CFF80132
:1028100081918F010E94A411F701819391937F010F
:10282000F3E0053B1F0799F78091F8038770BE011D
:102830006F5F7F4F45EE54E00E947C095D9A419A9C
:102840002091A5042223A1F09091DD03992381F02A
:102850008091A6048F5F8093A6048150821729F48B
:102860001092A604892F815001C0892F0E94A00BCD
:102870008091A4040E94CB0A80ED93E00E94EB08B3
:10288000682F84EE94E00E94910FE091A404EF5F22
:10289000E093A404E83131F0F0E0E053FC4F878589
:1028A000882341F41092A40405C05E9A409A89E0FE
:1028B0008093C0048091F803887171F180919A032C
:1028C000823051F58091BC049091BD04880F991F0E
:1028D0009093BD048093BC0483E080939A030E948C
:1028E000840C0E94252A6093B8047093B9048093E5
:1028F000BA049093BB04611571058105910561F4DB
:1029000081E090E0A0E0B0E08093B8049093B90437
:10291000A093BA04B093BB048091F80384FF1EC057
:102920008091BC049091BD048E7F0E943E0A182FB6
:102930008091B4046091BE040E947F0D082F8091A5
:10294000B504612F0E947F0D282F8091B6046091FD
:10295000B704402F00919B030E9410115D9841988D
:102960008091A7048130D1F0813020F0823009F0CD
:1029700047C034C082E10E94492B892B09F040C036
:1029800081E08093A7040E94172A6093A8047093A3
:10299000A9048093AA049093AB0432C082E10E9400
:1029A000492B892B21F50E94172A2091A8043091E8
:1029B000A9044091AA045091AB04621B730B840BD1
:1029C000950B695E734080409040D0F082E0809328
:1029D000A70480ED97E00E94DA1112C082E10E9404
:1029E000492B892B69F080E090E00E94DA11109267
:1029F000A70406C08091C004883009F058CF55CF95
:102A0000A096EAE00C94533083E161E00E94AA2A88
:102A100083E160E00E94162B82E08093B00085E0A5
:102A20008093B10083E061E00E94AA2A83E060E025
:102A30000E94162B08951F93182F0E94252A609339
:102A40009F047093A0048093A1049093A204109318
:102A50008D04112329F440E855E260E070E004C0E1
:102A600040E051EE60E070E089E396E00E94322E93
:102A70001F910895ACE1B0E0E0E4F5E10C9437304B
:102A80000E94252A7B018C0181E00E94A50B54E75E
:102A9000A52E6E010894C11CD11C43E0B42EA9825E
:102AA000C60161E00E94CD0FB0929A030E94840C8F
:102AB0006AEF70E080E090E00E944B2A80919A03D8
:102AC000833009F07DC089E396E00E94B92E892BFE
:102AD00009F076C00E94252A6E197F09800B910BA0
:102AE0006058734C894C914008F06AC0D8CF8FE78A
:102AF0000E94960A0E94AA0A843509F05CC0898364
:102B00000E94AA0A182F00E01093240400932304C3
:102B10000E94AA0A080F111D109324040093230495
:102B20000E94AA0A809322040E94AA0A8093210488
:102B3000813108F040C0FF2407C00E94AA0A0F5F3D
:102B40001B4FF8018083F3940F2D10E08091210436
:102B500090E0880F991F0817190778F380E7898399
:102B6000CE01019661E00E94CD0F83E080939A032D
:102B70000E94840C62E370E080E090E00E944B2AA7
:102B800080919A038330A9F08FE70E94960A0E94F1
:102B9000AA0A803581F4898305EB13E00E94AA0A12
:102BA000F80181938F01F3E0003D1F07B9F781E041
:102BB00003C082E001C083E06C96EAE00C945330DD
:102BC00080919A03833009F092CFF3CF83E00E9483
:102BD000BA0A8093F90384E00E94BA0A8093FA0348
:102BE00087E061E00E94C00A6AE070E080E090E067
:102BF0000E944B2A0E94840C000008950F931F939B
:102C0000082F19C05E9A409A64E670E080E090E078
:102C10000E944B2A5E98409864E670E080E090E065
:102C20000E944B2A1F5F101768F36CE271E080E08E
:102C300090E00E944B2A10E0F6CF482F392F25E074
:102C40000DC0F999FECF1FBA842F932F92BD81BD7D
:102C500060BD0FB6F894FA9AF99A0FBE215059F058
:102C6000F999FECF842F932F92BD81BDF89A80B53C
:102C7000681739F7089582E00E94FE150895A0E0D4
:102C8000B0E0E5E4F6E10C943030482E562EEE2408
:102C9000FF2488249924C0E0D0E0CC24DD2416E46D
:102CA000312E04C055245394CC24DD24442069F4EF
:102CB00080919B03839DE0011124BCE9EB2EB3E0DE
:102CC000FB2EA9E18A2E912C1DC021E0421671F441
:102CD00080919B03839DE00111246B96F0EDEF2E14
:102CE000F3E0FF2EE9E28E2E912C0CC032E0431669
:102CF00049F47BE9E72E73E0F72E61E0862E912CF4
:102D0000C8E1D1E03E016C0C7D1C1092360510929A
:102D10003505E3011BC0552059F4F999FECFD2BD0A
:102D2000C1BDF89A80B5F701E00FF11F808307C09D
:102D3000F701E00FF11FCE0160810E941D160E0DFC
:102D40001F1DF80180810E94300821969E012619DE
:102D5000022F10E008151905F0F2CE015520D9F424
:102D6000F999FECFD2BDC1BDF89A20B5F999FECF31
:102D70002196D2BDC1BD2197F89A80B590E0B22EC0
:102D8000AA248A299B2920913505309136052817D8
:102D9000390759F487CF2196609136050E941D1698
:102DA000CE01609135050E941D1680E291E0C80EAB
:102DB000D91E91EEC91692E0D90608F477CF852D79
:102DC000CDB7DEB7E1E10C944C3080E061E00E94C9
:102DD0003F1681E061E00E943F16089582E061E0C5
:102DE0000E943F16089582E060E00E943F168091A5
:102DF0009B03843020F010929B030E94EE160895EE
:102E00001F93182F0E94F31680919B03811731F0B6
:102E1000143020F410939B030E94EE161F91089526
:102E200010928B0485E6E6E2F4E0DF011D928A95BC
:102E3000E9F708951F93182F8F3711F08830E1F5C7
:102E4000E0918B04EE2309F455C0E150E0938B042C
:102E5000F0E0EA5DFB4F108289E396E06DE00E94AE
:102E60002C2F10E00AC0E12FF0E0EA5DFB4F89E370
:102E700096E060810E942C2F1F5F80918B041817B1
:102E800090F389E396E060E20E942C2F89E396E0BC
:102E90006DE00E942C2F10E00AC0E12FF0E0EA5D07
:102EA000FB4F89E396E060810E942C2F1F5F809189
:102EB0008B04181790F31CC08B3119F40E94101763
:102EC0001FC08D30E9F08A30D9F080918B048436B0
:102ED00088F489E396E0612F0E942C2F80918B0467
:102EE000E82FF0E0EA5DFB4F10838F5F80938B0447
:102EF00080E007C089E396E067E00E94E02BF8CF0E
:102F000081E01F9108951F93CF93DF93CFEDD3E01E
:102F100010E03BC089E396E062E271E00E94712D0F
:102F200089E396E0612F4AE050E00E94EE2C89E3AD
:102F300096E06FE271E00E94712D699170E080E08F
:102F400090E02091DE0330E040E050E00E94C02F8E
:102F500020E137E240E050E00E94C02FDC01CB01CD
:102F60004091D5035091D6036091D7037091D80357
:102F7000480F591F6A1F7B1F89E396E02AE030E063
:102F80000E94B52C1F5F183119F08881882311F633
:102F9000DF91CF911F910895EF92FF920F931F93AE
:102FA000882339F489E396E061E77AE00E94FE2BFA
:102FB0003BC090E00E94B20824E630E040E050E0E0
:102FC0000E94F22F122F032FF42EE52E622F732F63
:102FD000842F952F2AE030E040E050E00E94F22F4D
:102FE00089E396E0BA01A9012AE030E00E94A62C0C
:102FF00089E396E06EE20E94E02B612F702F8F2D07
:103000009E2D2AE030E040E050E00E94F22FAB011C
:10301000BC0189E396E02AE030E00E94A62C89E317
:1030200096E063E70E94122C1F910F91FF90EF90A2
:103030000895FF920F931F93CF93DF9389E396E058
:1030400067E67AE00E94BF2B8091B503813041F49E
:1030500089E396E06EE47AE00E94FE2BFF246DC0C7
:10306000823029F489E396E067E37AE0F5CF843093
:1030700029F489E396E063E27AE0EECF853071F7D8
:1030800089E396E068E17AE0E7CFCF2DD0E0C93060
:10309000D1051CF06F2D685C02C06F2D6F5C89E359
:1030A00096E00E94E02B89E396E060E17AE00E94DE
:1030B000BF2BBE016F5F7F4F89E396E04AE050E08F
:1030C0000E944A2D89E396E065E07AE00E94BF2BDA
:1030D0008E010B541C4FD8011196EC91E032F8F49C
:1030E00089E396E068EF79E00E94BF2BF8018181C7
:1030F000803130F089E396E063E371E00E94712D46
:10310000CB54DC4F698170E06F7070706F5F7F4FE0
:1031100089E396E04AE050E00E945D2D0DC0F0E0AA
:10312000EF70F070EE0FFF1FE75BFC4F6081718165
:1031300089E396E00E94742DF39480912204F8169E
:1031400008F4A3CF89E396E06DED79E00E94BF2BF0
:103150008091CD030E94CC1789E396E062EC79E080
:103160000E94BF2B8091CE030E94CC1789E396E08A
:1031700067EA79E00E94BF2B8091CF030E94CC17B1
:1031800089E396E06CE879E00E94BF2B4091C5038B
:103190005091C6036091C7037091C8034115510552
:1031A0006105710539F189E396E02AE030E00E947B
:1031B000B52C89E396E069E579E00E94BF2B809108
:1031C000C9030E94E508AB01BC0189E396E02AE04F
:1031D00030E00E94B52C89E396E065E379E00E9437
:1031E000BF2B89E396E06091CA034AE050E00E9459
:1031F000002D06C089E396E06CE279E00E94FE2B88
:1032000089E396E06FE079E00E94BF2B6091CB03E9
:103210007091CC0389E396E04AE050E00E94DA2CFA
:1032200089E396E062EF78E00E94BF2B6091C403CF
:10323000603450F470E06F5F7F4F89E396E04AE0BE
:1032400050E00E945D2D06C089E396E069EE78E0CB
:103250000E94FE2B89E396E06CEC78E00E94BF2B85
:103260008091C30380FD03C065E371E002C069E3A0
:1032700071E089E396E00E94742D89E396E06FEA9D
:1032800078E00E94BF2B8091C30382700E94890D59
:1032900089E396E060E978E00E94BF2B8091C30348
:1032A00084700E94890D89E396E061E778E00E94CE
:1032B000BF2B8091C30388700E94890DCDB7DEB704
:1032C000E5E00C9458301F93CF93DF9389E396E0A9
:1032D0006BEB7BE00E94BF2B4091D5035091D6034E
:1032E0006091D7037091D80389E396E02AE030E03B
:1032F0000E94B52C89E396E065EA7BE00E94BF2B33
:103300004091D9035091DA036091DB037091DC03A3
:1033100089E396E020E130E00E94B52C89E396E055
:103320006FE87BE00E94BF2B89E396E06091DD03AC
:103330004AE050E00E94002D89E396E069E77BE0D7
:103340000E94BF2B89E396E06091DE034AE050E0E3
:103350000E94002D89E396E063E67BE00E94BF2B8C
:10336000CFEDD3E010E012C0112331F089E396E0F5
:103370006DE371E00E94712D89E396E069914AE066
:1033800050E00E94EE2C1F5F183119F088818823CD
:1033900059F789E396E00E94E82B89E396E06DE413
:1033A0007BE00E94BF2B89E396E06091F7034AE03F
:1033B00050E00E94002D89E396E068E37BE00E94E4
:1033C000BF2BE091F803F0E0E770F070EE0FFF1F05
:1033D000E759FC4F6081718189E396E00E94742D6A
:1033E00089E396E063E27BE00E94BF2B8091F803C3
:1033F00090E0887190708830910589F0893091054E
:103400001CF4892B39F01BC08031910569F0489775
:10341000B1F40FC089E396E06AE17BE00EC089E376
:1034200096E06EE07BE009C089E396E068E07BE02F
:1034300004C089E396E06EEF7AE00E94FE2B89E3F8
:1034400096E06AEE7AE00E94BF2B4091D103509142
:10345000D2036091D3037091D40389E396E02AE00C
:1034600030E00E94B52C89E396E061ED7AE00E949D
:10347000BF2B8091A10380710E94890D89E396E0A2
:1034800068EB7AE00E94BF2B8091A10380740E94B8
:10349000890D89E396E06FE97AE00E94BF2B809165
:1034A000A10380720E94890D89E396E062E87AE0C8
:1034B0000E94BF2B80ED93E00E94F508AB01BC0198
:1034C00089E396E02AE030E00E94A62C89E396E0AA
:1034D0006DE77AE00E94BF2B80ED93E00E94F50833
:1034E0009B01AC0160E472E48FE090E00E94F22F57
:1034F00089E396E0BA01A9012AE030E00E94A62CF7
:1035000089E396E06AE77AE00E94FE2BDF91CF9193
:103510001F910895EF92FF920F931F937C0109E38F
:1035200016E0C8016F2D70E04AE050E00E94C92CFF
:10353000C8016EE20E94E02BB70124E07695679502
:103540002A95E1F76F707070C8014AE050E00E9460
:10355000C92CC8016EE20E94E02B8FE0E822FF2414
:10356000C801B7014AE050E00E94C92C1F910F9199
:10357000FF90EF9008950F931F93CF93DF932091C7
:1035800025042F3FA9F589E396E061EF75E00E94DD
:10359000BF2B83E793E00E948A1A89E396E060EDEF
:1035A00075E00E94BF2B80912304909124040E9417
:1035B0008A1A89E396E06DE975E00E94FE2B89E3A3
:1035C00096E06AE775E00E94FE2B89E396E062E6EA
:1035D00075E00E94FE2B89E396E06DE375E00E94A2
:1035E000FE2B89E396E00E94E82B0E94191869C01F
:1035F00012160CF066C0332727FD30958091220407
:1036000090E0821793070CF45CC089E396E068E2CF
:1036100075E00E94BF2B60912504772767FD7095A8
:1036200089E396E04AE050E00E945D2D89E396E050
:103630006DEF74E00E94BF2B08E210E03AC0C12F8A
:10364000D0E0CC0FDD1FCF5FDB4F288130E08091D1
:103650002504992787FD909501972817390741F58B
:1036600089E396E06FE371E00E94712D89E396E0B3
:10367000602F4AE050E00E94EE2C89E396E063E47C
:1036800071E00E94712DE981F0E0EF70F070EE0FB3
:10369000FF1FE75BFC4F6081718189E396E00E9428
:1036A000712D89E396E067E471E00E94712D0F5F50
:1036B0001F5F80912104181710F289E396E00E94A1
:1036C000E82BDF91CF911F910F910895ACE1B0E00D
:1036D000ECE6FBE10C943930282F809125048F3FD4
:1036E00009F03BC1822F90E0FC013A97EF36F105DB
:1036F00008F02CC1EC5CFF4F0C94663089E396E037
:1037000069E471E0A7C089E396E065E571E00E9495
:10371000742D85E78983DE011296E5EBF3E08BE1FA
:1037200001900D928150E1F7CE0101966CE10E946B
:10373000CD0F0E94840C83E080939A0368EC70E0C4
:1037400080E090E00E944B2A80919A03843009F037
:10375000FDC08FE70E94960A0E94AA0A89838535D8
:1037600009F0F4C089E396E06FED74E00E94FE2B4F
:1037700089E396E061EC74E00E94FE2B89E396E019
:1037800063EA74E0ACC089E396E06DE671E00E9404
:10379000742D89E68983CE01019661E00E94CD0FE8
:1037A0000E94840C83E080939A0368EC70E080E0D0
:1037B00090E00E944B2A80919A03843009F0C6C0A1
:1037C0008FE70E94960A0E94AA0A89838E010E5FE3
:1037D0001F4FBDE1EB2EF12CEC0EFD1E0E94AA0A3C
:1037E000D8018D938D01AE15BF05C1F7A5EBB3E0F0
:1037F000FE0132968BE101900D928150E1F78981B3
:10380000893409F0A3C089E396E065E874E00E947A
:10381000FE2B89E396E067E674E00E94FE2B89E3C5
:1038200096E069E474E05BC089E396E067E871E0E4
:103830000E94742D8EEF8093250488C0205227505B
:10384000922F905380912204891738F489E396E0EF
:1038500066E971E00E94742D79C0909325046FC0D1
:1038600084E18093250489E396E062E174E037C047
:1038700085E18093250489E396E06BED73E02FC02A
:1038800086E18093250489E396E064EA73E027C02B
:1038900087E18093250489E396E06AE573E01FC021
:1038A00088E18093250489E396E069E473E017C01A
:1038B00089E18093250489E396E065E373E00FC016
:1038C0008AE18093250489E396E060E273E007C013
:1038D0008BE18093250489E396E068EF72E00E9413
:1038E000FE2B34C089E396E06EED72E00E94FE2B61
:1038F0008091C30391E01DC089E396E068EC72E01B
:103900000E94FE2B8091C30392E013C089E396E0EE
:1039100063EB72E00E94FE2B8091C30394E009C028
:1039200089E396E068E972E00E94FE2B8091C30370
:1039300098E089278093C3038FEF809325040E942A
:10394000BB1A04C089E396E00E94F32E89E396E057
:103950000E94B92E892BB1F762C1822F0E941A17DB
:10396000882309F45CC180918B04882321F48FEFB4
:10397000809325044CC186E294E060E070E040E072
:1039800050E00E94A2069B01AC0160912504862FA5
:10399000992787FD9095A92FB92FFC013197EB311D
:1039A000F10508F024C1ED55FF4F0C946630E62F69
:1039B000FF27E7FDF0958091220490E08E179F0786
:1039C0000CF415C1DA01C9010197A109B109809769
:1039D000A105B10548F0A8E2FA2E00E010E06F0161
:1039E0000894C108D10825C0EB54FC4F822F8150A8
:1039F0008083E5C0612F70E0660F771F6F5F7B4F9C
:103A0000FB01808190E08C159D0591F48F2D90E055
:103A1000A0E0B0E082179307A407B50741F4F601D0
:103A2000EB54FC4FDB0111968C91818301E0F39400
:103A30001F5F809121041817E8F2BFC02F3F3105A6
:103A40004105510511F008F0D2C02093CD03B7C055
:103A50002F3F31054105510511F008F0C8C02093F2
:103A6000CE03ADC02F3F31054105510511F008F0DF
:103A7000BEC02093CF03A3C080912604806280370C
:103A800019F587E294E060E070E040E050E00E94C9
:103A9000A2069B01AC01DC01CB010197A109B10990
:103AA0000897A105B10508F0B5C0CA01B90124ED18
:103AB00030E340E050E00E94C02F9B01AC012A5E41
:103AC0003C4A4A46554E24C0863611F587E294E0BA
:103AD00060E070E040E050E00E94A2069B01AC0173
:103AE000DC01CB010197A109B1090797A105B10537
:103AF00008F090C0CA01B90128EA31E640E050E080
:103B00000E94C02F9B01AC01245E3C434E46544EA4
:103B1000211531054105510561F0DA01C9018050D7
:103B20009447AB48B24381509A45A246B24008F050
:103B30005EC02093C5033093C6034093C7035093E0
:103B4000C8033DC02F3F31054105510511F008F074
:103B50004EC02093C90333C0DA01C9010197A109FE
:103B6000B1098F3F9105A105B10508F040C0209330
:103B7000CA0325C0DA01C901845C9940A040B04065
:103B80008D549D41A040B04030F43093CC0320933D
:103B9000CB0301E001C000E02115310541055105CD
:103BA00011F48FEF07C0213431054105510528F488
:103BB000822F81508093C40302C00023C1F0809102
:103BC0008C048823D1F48091D9039091DA03A091D9
:103BD000DB03B091DC030196A11DB11D8093D903D5
:103BE0009093DA03A093DB03B093DC0306C089E370
:103BF00096E068EA71E00E94742D0E9410178FEF22
:103C00008093250489E396E06AE00E94122C0E94CA
:103C1000BB1A05C021E030E040E050E07ECF6C965A
:103C2000E8E00C94553089E396E06CE472E00E9481
:103C3000FE2B89E396E064E372E00E94FE2B89E3A9
:103C400096E00E94B92E892B31F089E396E00E941C
:103C5000F32E0E94661B0E943A15823019F08330C1
:103C600069F405C089E396E066E172E004C089E387
:103C700096E06FEF71E00E94FE2B08958FEF809326
:103C8000250410928C040E94BB1A0CC089E396E0B4
:103C90000E94B92E892B31F089E396E00E94F32E21
:103CA0000E94661B809125048E3F81F708958091C4
:103CB0002504992787FD9095A92FB92FFC013196EE
:103CC000EB30F10508F074C0E254FF4F0C946630FD
:103CD00089E396E064E678E00E94FE2B83E793E0B8
:103CE0000E948A1A89E396E06CE478E00E94FE2B39
:103CF00089E396E067E278E00E94FE2B89E396E094
:103D00006DEF77E00E94FE2B89E396E06CED77E0A3
:103D10000E94FE2B89E396E06FEA77E00E94FE2B7B
:103D200089E396E069E877E00E94FE2B89E396E05C
:103D300065E677E00E94FE2B89E396E06EE377E08C
:103D40000E94FE2B89E396E00E94E82B0E946319F3
:103D50002FC089E396E061E277E028C089E396E02E
:103D60006CEF76E023C089E396E067EE76E01EC054
:103D700089E396E068EC76E019C089E396E064E8B0
:103D800076E014C089E396E06FE676E00FC089E341
:103D900096E06AE576E00E94FE2B89E396E064E116
:103DA00076E004C089E396E06EEF75E00E94FE2B9A
:103DB0006AE070E080E090E00E944B2A04C089E352
:103DC00096E00E94F32E89E396E00E94B92E892B9B
:103DD000B1F70895A2E2B0E0E0EFFEE10C942F30DD
:103DE0008E010F5F1F4F80E1D8011D928A95E9F780
:103DF00089E396E066EC71E00E94742D0E94E6155E
:103E000020E034E74BE852E32F8F38A349A35AA3AD
:103E100080E09EECADEEB4E38B8F9C8FAD8FBE8FB8
:103E200024EF31E040E050E02F8B388F498F5A8FDC
:103E300030E5C32E33ECD32EE12CF12C412C24E7BA
:103E4000522E2BE8622E22E3722E882499245401EC
:103E500033241E8A1D8A198A1A8A1B8A1C8AFFC06B
:103E600089E396E00E94F32E8434B9F0853430F46F
:103E70008332B9F18C3209F0CCC044C0833509F0EB
:103E8000C8C02F8D38A149A15AA1C901DA012C015E
:103E90003D01882499245401E2C089E396E064E45A
:103EA0000E94E02B89E396E040E054E76BE872E380
:103EB0002AE030E00E94142D89E396E06CE20E9433
:103EC000E02B89E396E040E05EEC6DEE74E32AE0DF
:103ED00030E00E94142D89E396E06CE20E94122CDF
:103EE000BEC019821A821B821C821D821E821F8202
:103EF000188619861A861B861C861D861E861F86B6
:103F0000188A3AC0339434E0331609F0A8C06981A6
:103F10007A818B819C8128EE33E040E050E00E9462
:103F2000C02F6F8F78A389A39AA36D817E818F8123
:103F300098850E94C02F6B8F7C8F8D8F9E8F898577
:103F40009A85AB85BC858F8B988FA98FBA8F6D852D
:103F50007E858F8598890E94C02F6B017C0190E23D
:103F6000C9169EE4D90690E0E90690E0F90630F41F
:103F70008CE162E30E94C00A332471C0A0E3CA1638
:103F8000A5E7DA06A0E0EA06A0E0FA0618F48CE15C
:103F900062E2F0CFB0E4CB16BCE9DB06B0E0EB06A2
:103FA000B0E0FB0618F48CE166E2E4CFE0E5CE1663
:103FB000E3ECDE06E0E0EE06E0E0FE0618F48CE15D
:103FC00062E1D8CFF0E6CF16FAEEDF06F0E0EF06BA
:103FD000F0E0FF0618F48CE165E1CCCF20E7C216D3
:103FE00021E1D20621E0E20620E0F20618F48CE19D
:103FF00061E0C0CF30EAC31636E8D30631E0E3060D
:1040000030E0F30618F48CE163E0B4CF8CE165E0B6
:10401000B1CF90ED292E280E49E0421500F1032D75
:1040200010E0000F111F000F111F81E090E08C0FB6
:104030009D1F080F191FD8016D917D918D919C9145
:104040002AE030E040E050E00E94C02F620D711D78
:10405000811D911DF801608371838283938389E3BD
:1040600096E00E94B92E892B09F0FACE81149104B2
:10407000A104B10489F4C301B2010E94360B61E0CE
:1040800070E080E090E00E944B2AFFEFFE8B1D8ADB
:10409000198A1A8A1B8A1C8A2F89388D498D5A8D54
:1040A00082169306A406B506E0F40E94E10A298967
:1040B0003A894B895C89280F311D411D511D298B7F
:1040C0003A8B4B8B5C8B3D89381708F48D8B4E896E
:1040D000841708F48E8B0894811C911CA11CB11CC0
:1040E00056C0C301B20128EE33E040E050E00E9428
:1040F000F22F89E396E0BA01A9012AE030E00E949C
:10410000A62C89E396E06CE20E94E02B89E396E01E
:104110006D894AE050E00E94EE2C89E396E06CE263
:104120000E94E02B69897A898B899C89A501940179
:104130000E94F22F89E396E0BA01A9012AE030E05B
:104140000E94A62C89E396E06CE20E94E02B89E3B2
:1041500096E06E894AE050E00E94EE2C89E396E0FA
:104160006CE20E94122C4C0C5D1C6E1C7F1C8B8D13
:104170009C8DAD8DBE8D84159505A605B70520F4E3
:104180004F8C58A069A07AA08824992454012F8DBF
:1041900038A149A15AA1285E33404040504009F05F
:1041A0005ECFA296E2E10C944B30A0E0B0E0EBEDE4
:1041B000F0E20C943A300E94252A611571058105C0
:1041C0009105C9F30E9499061092D9031092DA035F
:1041D0001092DB031092DC03DD24E090D903F09011
:1041E000DA030091DB031091DC03102F0F2DFE2C5E
:1041F000EE240E9494062FEF30E040E050E00E9451
:104200001430E60EF71E081F191FE092D903F09232
:10421000DA030093DB031093DC03D39444E0D41659
:10422000E1F6CFEDD3E000E010E040E1E42E47E21C
:10423000F42E4EC00F5F19F40E944D084DC00E942D
:10424000940622E330E040E050E00E9414306F5FBB
:10425000EFEDF3E090E004C08191861759F39F5F82
:104260009117D0F38091DE0390E08E9D90018F9D99
:10427000300D9E9D300D1124862F90E0AC01249FBF
:10428000C001259F900D349F900D1124AA2797FD02
:10429000A095BA2F2091D5033091D6034091D70332
:1042A0005091D803820F931FA41FB51F20919D0327
:1042B00030919E0340919F035091A0032817390726
:1042C0004A075B0708F4B6CF69931F5F183121F0E6
:1042D0008881882309F0AECFCDB7DEB7E7E00C9434
:1042E000563080E060E00E943F16882331F081E084
:1042F00060E00E943F16882341F40E9492080E94C9
:104300004D080E94D5200E94E5160895AAE5B0E068
:10431000ECE8F1E20C943B308B017A018B3009F42C
:1043200026C18C3040F5853009F484C0863080F495
:10433000823009F459C0833020F4813009F050C232
:1043400042C0833009F461C0843009F049C265C0BD
:10435000883009F49DC0893038F4863009F486C06D
:10436000873009F03DC28CC0893009F499C08A3089
:1043700009F036C2C9C0893609F482C18A3680F490
:10438000863609F42DC1873620F4853609F028C217
:104390000EC1873609F43DC1883609F021C241C1FA
:1043A0008C3609F4C4C18D3638F48A3609F473C1E9
:1043B0008B3609F015C2AFC18D3609F4ECC1873CCC
:1043C00009F00EC200C281E069E270E00E9485112E
:1043D00000ED13E0F80181918F010E946E11F3E06E
:1043E000093F1F07B9F704C282E06BE170E00E9449
:1043F000851105EB13E0F80181918F010E946E1188
:10440000F3E0003D1F07B9F7F3C183E061E070E01E
:104410000E9485110E943A15E9C184E061E070E0D4
:104420000E94851181E00E946E110E9467110E9416
:10443000EA1EE0C16091210470E0660F771F85E0FD
:104440000E94851100E010E008C0F801EF5FFB4F0B
:1044500080810E946E110F5F1F4F8091210490E0B8
:10446000880F991F0817190780F3C2C186E062E020
:1044700070E00E94851183E793E00E947C11B8C12F
:1044800087E061E070E00E94851180912204AEC156
:1044900088E061E070E00E94851180919B03A6C1D5
:1044A00086E68983CE01019661E00E94CD0F0E94CD
:1044B000840C83E080939A0368EC70E080E090E0E5
:1044C0000E944B2A80919A038430E1F48FE70E9486
:1044D000960A0E94AA0A8983863471F489E060E210
:1044E00070E00E94851110E00E94AA0A0E946E11DD
:1044F0001F5F1032C9F77CC189E061E070E00E9463
:104500008511C7C089E06DC18AE069E170E00E9451
:10451000851181E080939C038091A305882351F04D
:104520008091A1039091A203A091A303B091A40351
:10453000806809C08091A1039091A203A091A30378
:10454000B091A4038F778093A1039093A203A093CB
:10455000A303B093A4030CE913E0F80181918F0148
:104560000E946E11F3E0053B1F07B9F741C18BE0D4
:1045700061E270E00E9485118091C0048F3F39F0A4
:104580008091C0048F5F8093C004815002C08091ED
:10459000C0040E946E1110E0812F0E94A4110E949D
:1045A000190A0E947C111F5F1031B1F721C185E605
:1045B00061E070E00E9485110932110509F015C112
:1045C00020E030E0F901E053FC4FD701A20FB31F08
:1045D0008C9180832F5F3F4F2932310599F759C065
:1045E00086E661E070E00E9485110B31110509F04B
:1045F000FCC020E030E0F901EB54FC4FD701A20FE2
:10460000B31F8C9180832F5F3F4F2B31310599F77A
:1046100040C087E661E070E00E9485110E94E516C7
:1046200038C088E661E070E00E94851185E78A83E2
:10463000DE011396E5EBF3E08BE101900D928150E2
:10464000E1F7CE0102966CE10E94CD0F0E94840C2E
:1046500083E080939A0360E273E080E090E00E9440
:104660004B2A80919A03843009F0BFC08FE70E94E3
:10467000960A0E94AA0A8A83853509F0B6C009C045
:1046800089E661E070E00E9485110E944D080E9459
:10469000920881E0ABC08AE661E070E00E9485117B
:1046A00089E68E8FCE014E9661E00E94CD0F0E946A
:1046B000840C83E080939A0360E273E080E090E0F2
:1046C0000E944B2A80919A03843009F08EC08FE7B4
:1046D0000E94960A0E94AA0A8E8F8E01015E1F4FC9
:1046E0006AE3E62EF12CEC0EFD1E0E94AA0AF801E8
:1046F00081938F01EE15FF05C1F7A5EBB3E0FE0135
:104700007F968BE101900D928150E1F78E8D893477
:1047100009F06BC0BECF8BE661E070E00E948511AE
:10472000F70180810E9400170E947121B2CF8CE6B0
:1047300061E070E00E9485110032110571F487E696
:104740008AAFDE01DB96F70180E201900D92815085
:10475000E1F7CE01CA9661E205C087E48AAFCE01D7
:10476000CA9661E00E94CD0F0E94840C83E0809382
:104770009A036CE474E080E090E00E944B2A809100
:104780009A03843091F58FE70E94960A0E94AA0A44
:10479000873459F57ECF8DE661E070E00E94851187
:1047A0000931110511F520E030E0F901E456FC4F24
:1047B000D701A20FB31F8C9180832F5F3F4F293108
:1047C000310599F766CF87EC61E070E00E948511B2
:1047D00081E00E946E110E9467111092FF030AC0CF
:1047E0008AEC61E070E00E94851180E00E946E1109
:1047F0000E946711C65ADF4FE6E00C945730A0E0E4
:10480000B0E0E5E0F4E20C94373084E0A82E06E056
:10481000B02E15E0C12E07E315E0B4E6DB2EA2E0D2
:10482000EA2EF3E0FF2EA1C089E396E00E94F32E6A
:10483000982F8093A2058091A105833021F18430C7
:1048400028F4813099F08230B8F409C0853009F439
:1048500048C0853020F1863009F087C05FC0953BA5
:1048600009F083C081E08093A1057FC0923609F0F2
:104870007AC0E092A10579C09093A00590939F051E
:10488000F092A10572C090939D0510929E058091B3
:104890009F05892780939F05A092A10566C0D92F07
:1048A000C0E020919D0530919E052C2B3D2B30932F
:1048B0009E0520939D0580919F05892780939F05E4
:1048C000C092A1052536310508F44FC08CEC61E09B
:1048D00070E00E94851181E00E946E110E946711B4
:1048E00042C020919B0530919C05F901E95CFA4F8B
:1048F000908380919F05892780939F052F5F3F4F6D
:1049000030939C0520939B0580919D0590919E0579
:104910002817390750F1B092A10527C080919F0553
:10492000891759F460919B0570919C058091A005B1
:1049300047E355E00E9486210DC08BEC62E070E0F9
:104940000E9485118091A0050E946E118091000443
:104950000E946E11F8018D2D11928A95E9F710923F
:104960009C0510929B051092A10589E396E00E9498
:10497000B92E892B09F058CFCDB7DEB7EAE00C94F9
:10498000533081E08093FF0308C089E396E00E94E2
:10499000B92E892B11F00E94FF238091FF038823F9
:1049A000A1F708951F93109125041F3F09F0F1C04E
:1049B000893409F467C08A3428F5883309F479C04A
:1049C000893368F4803309F486C0813308F06FC0FE
:1049D0008B3109F44DC0813209F0D5C03DC081341E
:1049E00009F49AC0823438F4893309F472C08034EF
:1049F00009F0C9C031C0823409F4A1C0863409F07D
:104A0000C2C052C0823609F49AC0833690F4883509
:104A100079F1893538F4823509F43FC0833509F0DE
:104A2000B2C01FC08A3509F4A9C0813609F0ABC0F5
:104A300073C0823791F1833730F48636A9F1893615
:104A400009F0A1C01FC0883799F08A3709F496C0D1
:104A5000833709F098C005C089E396E069E471E006
:104A600019C00E94E51689E396E063ED71E006C087
:104A70000E94712189E396E06DEE71E00E94742D31
:104A80008EEF7FC00E944D080E94920889E396E055
:104A90006CE072E00E94742D76C00E94D52089E3FC
:104AA00096E065E272E0F6CF0E9483176CC08053F7
:104AB00068C089E396E06CEE71E00E94FE2B909155
:104AC000F803892F885F8871977E892B8093F8037C
:104AD00020C089E056C089E396E069ED71E00E944C
:104AE000FE2B8091A1039091A203A091A303B0910A
:104AF000A40320E130E040E050E082279327A42780
:104B0000B5278093A1039093A203A093A303B0932E
:104B1000A4031093250437C089E396E063EC71E0A9
:104B20000E94FE2B8091A1039091A203A091A30368
:104B3000B091A40320E430E040E050E012C089E3EB
:104B400096E062EB71E00E94FE2B8091A1039091B0
:104B5000A203A091A303B091A40320E230E040E0BF
:104B600050E082279327A427B5278093A103909331
:104B7000A203A093A303B093A40302C00E94131E38
:104B80008FEF80932504809125048E3F09F4DDC0CA
:104B9000D4C00E941A17882309F4D7C080918B04CF
:104BA000882321F48FEF80932504C7C086E294E028
:104BB00060E070E040E050E00E94A2069B01AC0182
:104BC00080912504992787FD9095A92FB92FFC0185
:104BD0003197E930F10508F08CC0E753FF4F0C9492
:104BE0006630DA01C90181509447AB48B2438F5F08
:104BF0009945A246B24008F07CC02093D50330937B
:104C0000D6034093D7035093D8039AC02093D90377
:104C10003093DA034093DB035093DC0381E080930D
:104C20008C048EC0283031054105510508F061C063
:104C30002093DD0385C0DA01C9010197A109B109FB
:104C40000A97A105B10508F054C02093DE0378C08F
:104C500086E294E06DE371E00E94BE0710E00EC0B2
:104C6000183130F4E12FF0E0E053FC4F87871F5FED
:104C700080E090E06DE371E00E94BE07009759F07C
:104C80000E94A007009761F706C0E12FF0E0E05313
:104C9000FC4F17861F5F1831C0F352C02530310515
:104CA0004105510530F52093F7034AC0DA01C901E7
:104CB0000197A109B1090697A105B105D0F480912A
:104CC000F803887F822B8093F8033AC0DA01C90188
:104CD0000197A109B1098050924CA140B04048F41D
:104CE0002093D1033093D2034093D3035093D40342
:104CF00027C089E396E068EA71E00E94742D13C032
:104D00008091D9039091DA03A091DB03B091DC0389
:104D10000196A11DB11D8093D9039093DA03A0934E
:104D2000DB03B093DC030E9410178FEF8093250400
:104D300089E396E06AE00E94122C0E94571E05C08B
:104D400080918C048823E1F2EECF1F9108958FEFBC
:104D50008093250410928C040E94571E0CC089E396
:104D600096E00E94B92E892B31F089E396E00E94EB
:104D7000F32E0E94D224809125048E3F81F76AE0B1
:104D800070E080E090E00E944B2A04C089E396E046
:104D90000E94F32E89E396E00E94B92E892BB1F789
:104DA0000895AAE2B0E0E7EDF6E20C9434300E94F8
:104DB000172A7B018C0181E00E94A50B04C089E3C6
:104DC00096E00E94F32E89E396E00E94B92E892B8B
:104DD000B1F75E984098DD24D39432E6732E22E03A
:104DE000822E912C8C0E9D1E5E010894A11CB11C7C
:104DF00093E0C92E0E94172A20E030E06E197F0947
:104E0000800B910B693C71058105910510F021E043
:104E100030E08D2D90E028233923232BA9F10E9427
:104E2000172A7B018C015D9A419A80ED97E00E94E0
:104E3000DA117982D401E0EDF3E089E201900D927C
:104E40008150E1F7C5016AE20E94CD0F5D9841985B
:104E500080E090E00E94DA11C0929A030E94840CD4
:104E600062E370E080E090E00E944B2A80919A0318
:104E7000843051F4C0929A038FE70E94960A0E94F0
:104E8000AA0A823409F4DD2482E10E94492B892B8D
:104E900069F5DD24D3942AC05E9A409A5D9A419ABE
:104EA00089E396E00E94F32E8D30910569F08E30F3
:104EB00091051CF40A97B1F407C08332910569F09B
:104EC0008234910579F40CC089E396E064EA71E0DC
:104ED0000E94FE2B0E94A72605C00E94EA1E02C067
:104EE0000E94C1245E9840985D98419889E396E0BD
:104EF0000E94B92E892B09F47DCFCECF8F929F923D
:104F0000AF92BF92CF92DF92EF92FF920F931F93D7
:104F100082E10E94492B892B09F083C068EC70E084
:104F200080E090E00E944B2A80E090E00E94DA113D
:104F30000E94172A5B016C0140ECE42E42E1F42E42
:104F4000012D112DE60EF71E081F191F06C082E164
:104F50000E94492B892B09F062C00E94172A6E1506
:104F60007F058007910798F382E10E94492B892BE6
:104F700009F055C080ED97E00E94DA110E94172ACF
:104F80007B018C0199249394882488E496E2A0E024
:104F9000B0E0A80EB91ECA1EDB1E29C0AE14BF04A5
:104FA000C006D10638F480ED97E00E94DA1188241B
:104FB00083941DC00E94172A6E197F09800B910BE4
:104FC000693C71058105910590F00E94172A7B01CB
:104FD0008C0180E0992009F481E0982E882319F44F
:104FE00080E090E002C080ED97E00E94DA1182E15B
:104FF0000E94492B892B91F280E090E00E94DA1107
:10500000882049F080919B038F5F83700E94001776
:105010000E94712106C00E94D5200E94E5160E94C0
:10502000D1261F910F91FF90EF90DF90CF90BF900E
:10503000AF909F908F90089580E06DEF77E042E011
:1050400050E00E9452290895EF92FF920F931F9310
:1050500080E00E9419080E94C51186E061E00E946C
:10506000AA2A85E061E00E94AA2A8EE061E00E94FF
:10507000AA2A8FE061E00E94AA2A82E160E00E94F1
:10508000AA2A88E060E00E94AA2A88E061E00E94E3
:10509000162B0E94041589E396E040E052EC61E093
:1050A00070E00E94322E0E94F3160E9471210E942D
:1050B000640D8FEF8093C0040E941C2878940E9496
:1050C000172A7B018C018091C0048F3F09F0DFC05B
:1050D0000E94172A6E197F09800B910B605D774043
:1050E0008040904008F0D3C0EECF89E396E00E9464
:1050F000F32E89E396E00E94B92E892BB1F789E35C
:1051000096E062E472E00E94712D83E793E00E94D2
:105110008A1A89E396E069E572E00E94712D89E3BD
:1051200096E065E070E04AE050E00E945D2D62E3A9
:1051300070E080E090E00E944B2A89E396E00E94B4
:10514000B92E04970CF189E396E00E94F32E823485
:105150009105D1F489E396E00E94F32E8E349105F7
:1051600099F489E396E00E94F32E8434910561F46A
:1051700089E396E00E94F32E819731F480E090E07D
:105180000E94DA110E94D1264091D1035091D2039E
:105190006091D3037091D403DB01CA010197A10987
:1051A000B1090497A105B10568F44093C1044330E7
:1051B00029F040E052EC61E070E004C040EA56E8BB
:1051C00061E070E089E396E00E94322E0E947E2723
:1051D0005E98409880E090E00E94DA110E94640D91
:1051E0001092A5048091A10383FF11C08091E50373
:1051F000882351F08091EC03882331F08091F303F0
:10520000882311F087E001C085E08093A50480E049
:105210000E94A50B8091A4040E94CB0A0E94840CDA
:1052200010922B0510922C0510922D0510E015C040
:1052300062E370E080E090E00E944B2A80ED97E00E
:105240000E94DA1162E370E080E090E00E944B2A55
:1052500080E090E00E94DA111F5F80919B0381172C
:1052600038F78091F80390E084FF09C020E088714E
:105270009070489709F421E0822F0E941B158FE05F
:105280000E9419081F910F91FF90EF90089580EDF3
:1052900097E00E94DA1182E161E00E94162B5E9A8B
:1052A000409A27CF823000F5E82FF0E0EE0FFF1F85
:1052B000EC55FA4F71836083882319F08130A1F493
:1052C00008C0809169008C7F842B80936900E89AE4
:1052D000089580916900440F551F440F551F837F27
:1052E000842B80936900E99A08951F920F920FB65C
:1052F0000F9211242F933F934F935F936F937F935C
:105300008F939F93AF93BF93EF93FF938091A405E7
:105310009091A505892B29F0E091A405F091A505B0
:105320000995FF91EF91BF91AF919F918F917F91DF
:105330006F915F914F913F912F910F900FBE0F9002
:105340001F9018951F920F920FB60F9211242F9352
:105350003F934F935F936F937F938F939F93AF93FD
:10536000BF93EF93FF938091A6059091A705892B9A
:1053700029F0E091A605F091A7050995FF91EF911D
:10538000BF91AF919F918F917F916F915F914F915D
:105390003F912F910F900FBE0F901F9018951F9265
:1053A0000F920FB60F9211242F933F938F939F93D9
:1053B000AF93BF938091AC059091AD05A091AE05E0
:1053C000B091AF053091B0050196A11DB11D232FFD
:1053D0002D5F2D3720F02D570196A11DB11D209373
:1053E000B0058093AC059093AD05A093AE05B09346
:1053F000AF058091A8059091A905A091AA05B0914B
:10540000AB050196A11DB11D8093A8059093A90538
:10541000A093AA05B093AB05BF91AF919F918F91D7
:105420003F912F910F900FBE0F901F9018958FB73F
:10543000F8942091AC053091AD054091AE055091A6
:10544000AF058FBFB901CA0108959FB7F8942091A5
:10545000A8053091A9054091AA055091AB0586B5E4
:10546000A89B06C08F3F21F02F5F3F4F4F4F5F4FEC
:105470009FBF542F432F322F2227280F311D411D4C
:10548000511D82E0220F331F441F551F8A95D1F70B
:10549000B901CA010895EF92FF920F931F93CF9322
:1054A000DF937B018C010E94252AEB010EC00E9434
:1054B000252A6C1B7D0B685E7340C8F30894E108D5
:1054C000F10801091109C851DC4FE114F10401058B
:1054D000110569F7CDB7DEB7E6E00C945730789444
:1054E00084B5826084BD84B5816084BD85B58260E9
:1054F00085BD85B5816085BDEEE6F0E08081816087
:105500008083E1E8F0E01082808182608083808186
:1055100081608083E0E8F0E0808181608083E1EB5E
:10552000F0E0808184608083E0EBF0E08081816046
:105530008083EAE7F0E080818460808380818260FC
:1055400080838081816080838081806880831092E5
:10555000C1000895CF93DF93482F50E0CA018D5FBB
:10556000934FFC0134914151544FFA0184918823A7
:1055700069F190E0880F991FFC01EF52F44FA5915B
:10558000B491FC01E552F44FC591D491662351F4D6
:105590002FB7F8948C91932F909589238C938881C1
:1055A00089230BC0623061F42FB7F8948C91932F4C
:1055B000909589238C938881832B88832FBF06C085
:1055C0009FB7F8948C91832B8C939FBFDF91CF91E1
:1055D0000895833071F0843028F48130A1F0823056
:1055E00021F514C08630B1F08730D1F08430E9F471
:1055F00004C0809180008F7703C0809180008F7DF0
:1056000080938000089584B58F7702C084B58F7D24
:1056100084BD08958091B0008F778093B000089585
:105620008091B0008F7D8093B0000895FF920F931A
:105630001F93F62E482F50E0CA01895E934FFC015C
:105640002491CA018D5F934FFC0114914151544F35
:10565000FA0104910023C9F0222319F0822F0E943D
:10566000E92AE02FF0E0EE0FFF1FE552F44FA5917D
:10567000B4919FB7F894FF2021F48C911095812369
:1056800002C08C91812B8C939FBF1F910F91FF9033
:1056900008950F931F93482F50E0CA01895E934FDE
:1056A000FC012491CA018D5F934FFC01049141518B
:1056B000544FFA011491112319F420E030E015C081
:1056C000222319F0822F0E94E92A812F90E0880F6F
:1056D000991F8B51944FFC01A591B4918C9120E0BE
:1056E00030E0802311F021E030E0C9011F910F91DB
:1056F0000895982F8E3008F09E509770809148033F
:105700008295880F880F807C892B80937C00809104
:105710007A00806480937A0080917A0086FDFCCFC5
:105720002091780040917900942F80E030E0282B80
:10573000392BC9010895A0E0B0E0E1EAFBE20C9446
:1057400039307C016B018A01C0E0D0E00FC0D60186
:105750006D916D01D701ED91FC910190F081E02DEB
:10576000C7010995C80FD91F015010400115110537
:1057700071F7CE01CDB7DEB7E8E00C945530EF926B
:10578000FF920F931F93CF93DF937C018B01C0E0B7
:10579000D0E0F8010F5F1F4F6491662359F0D701E5
:1057A000ED91FC910190F081E02DC7010995C80FA2
:1057B000D91FEFCFCE01CDB7DEB7E6E00C9457305E
:1057C000DC01ED91FC910190F081E02D09950895A7
:1057D000EF92FF920F931F938C016DE00E94E02BDC
:1057E0007C01C8016AE00E94E02B9C012E0D3F1D48
:1057F000C9011F910F91FF90EF900895EF92FF92D2
:105800000F931F937C010E94BF2B8C01C7010E9444
:10581000E82B9C01200F311FC9011F910F91FF90B0
:10582000EF900895EF92FF920F931F937C010E94D7
:10583000E02B8C01C7010E94E82B9C01200F311F37
:10584000C9011F910F91FF90EF900895CF93DF93BF
:10585000EC016115710519F420E030E00FC0DB01A7
:105860000D900020E9F71197A61BB70BE881F9818D
:105870000280F381E02DAD0109959C01C901DF9102
:10588000CF9108954F925F927F928F929F92AF92A5
:10589000BF92CF92DF92EF92FF920F931F93DF930D
:1058A000CF93CDB7DEB7A1970FB6F894DEBF0FBE8A
:1058B000CDBF2C01742ECB01223008F42AE019A2AE
:1058C00031E2C32ED12CCC0EDD1E822E9924AA24C7
:1058D000BB24672D752FA50194010E94F22F790139
:1058E0008A01C801B701A50194010E94C02F472D6C
:1058F000461B0894C108D1084A3010F4405D01C02D
:10590000495CF6014083E114F1040105110521F021
:105910007E2C5F2DC801DDCFC201B6010E94262C6E
:10592000A1960FB6F894DEBF0FBECDBFCF91DF9129
:105930001F910F91FF90EF90DF90CF90BF90AF90AD
:105940009F908F907F905F904F900895DC0121157C
:10595000310541F4ED91FC910190F081E02D642F2F
:10596000099508950E94422C0895EF92FF920F939B
:105970001F937C010E94A62C8C01C7010E94E82B7A
:105980009C01200F311FC9011F910F91FF90EF90D3
:105990000895EF92FF920F931F939A017B0100E00D
:1059A00010E0B801A7010E94A62C1F910F91FF9053
:1059B000EF900895EF92FF920F931F937C010E9446
:1059C000C92C8C01C7010E94E82B9C01200F311FBC
:1059D000C9011F910F91FF90EF900895EF92FF92F0
:1059E0000F931F939A01E62EFF2400E010E0B80108
:1059F000A7010E94A62C1F910F91FF90EF90089590
:105A0000EF92FF920F931F937C010E94EE2C8C016A
:105A1000C7010E94E82B9C01200F311FC9011F9173
:105A20000F91FF90EF900895A0E0B0E0EAE1FDE271
:105A30000C943930EC016A017B012115310541F4E8
:105A4000E881F9810190F081E02D642F09951BC058
:105A50002A303105B1F477FF13C06DE20E94E02BCC
:105A60008C0144275527BA014C195D096E097F093D
:105A7000CE012AE00E94422C9C01200F311F04C05D
:105A80002AE00E94422C9C01C901CDB7DEB7E8E0B4
:105A90000C945530EF92FF920F931F937B019A0164
:105AA0000027F7FC0095102FB801A7010E94142DC4
:105AB0001F910F91FF90EF900895EF92FF920F9337
:105AC0001F937C010E944A2D8C01C7010E94E82B84
:105AD0009C01200F311FC9011F910F91FF90EF9082
:105AE00008950E94262C0895EF92FF920F931F9322
:105AF0007C010E94712D8C01C7010E94E82B9C0142
:105B0000200F311FC9011F910F91FF90EF90089551
:105B100008951F920F920FB60F9211242F933F9367
:105B20004F938F939F93EF93FF938091C00082FDDB
:105B30001DC04091C6002091F1053091F2052F5F04
:105B40003F4F2F7330708091F3059091F405281723
:105B5000390771F0E091F105F091F205EF54FA4F39
:105B600040833093F2052093F10502C08091C60076
:105B7000FF91EF919F918F914F913F912F910F90B6
:105B80000FBE0F901F9018951F920F920FB60F9295
:105B900011242F933F938F939F93EF93FF93209123
:105BA00035063091360680913706909138062817D1
:105BB000390731F48091C1008F7D8093C10014C0FA
:105BC000E0913706F0913806EB50FA4F2081809132
:105BD00037069091380601968F739070909338062F
:105BE000809337062093C600FF91EF919F918F918C
:105BF0003F912F910F900FBE0F901F901895A0E02E
:105C0000B0E0E5E0FEE20C943530FC011382128234
:105C100088EE93E0A0E0B0E084839583A683B78309
:105C20008BE893E0918380837587648757874687E5
:105C3000318B208B138B028BF58AE48AD78AC68A34
:105C4000B18EA08E938E828E8F85848F8889858F6A
:105C50008989868F8A89878F8B8980A32096ECE03B
:105C60000C945130AF92BF92DF92EF92FF920F935C
:105C70001F93CF93DF93EC017A018B01DD24403039
:105C800081EE580780E0680780E0780711F0DD2496
:105C9000D39491E0A92EB12CEC89FD89DD2069F027
:105CA000C50108A002C0880F991F0A94E2F78083FB
:105CB00060E079E08DE390E005C0108260E874E870
:105CC0008EE190E0A80197010E94F22F2150304010
:105CD00040405040569547953795279580E12030B4
:105CE000380720F0DD2011F0DD24D6CFE889F989CE
:105CF0003083EA89FB89208319A2EE89FF894081DC
:105D000021E030E0C9010C8C02C0880F991F0A9471
:105D1000E2F7482B4083EE89FF894081C9010D8C51
:105D200002C0880F991F0A94E2F7482B4083EE893E
:105D3000FF894081C9010E8C02C0880F991F0A9407
:105D4000E2F7482B4083EE89FF8980810F8C02C0E7
:105D5000220F331F0A94E2F7209528232083DF9136
:105D6000CF911F910F91FF90EF90DF90BF90AF9078
:105D70000895DC011C96ED91FC911D97E05CFF4FAE
:105D80002191319180819181281B390B2F733070C3
:105D9000C901089589E396E00E94B92E892B11F07C
:105DA0000E94882D0895DC011C96ED91FC911D97B1
:105DB000E05CFF4F20813181E054F040DF01AE5BB9
:105DC000BF4F8D919C9111972817390719F42FEF28
:105DD0003FEF07C08D919C91E80FF91F8081282F1C
:105DE00030E0C9010895DC011C96ED91FC911D97EE
:105DF000E05CFF4F20813181E054F040DF01AE5B79
:105E0000BF4F8D919C9111972817390719F42FEFE7
:105E10003FEF10C08D919C911197E80FF91F2081E1
:105E20008D919C91119701968F73907011969C9310
:105E30008E9330E0C9010895DC0191968C91919781
:105E4000882339F05496ED91FC915597808186FF17
:105E5000F9CF91961C920895CF93DF93EC01EE85D4
:105E6000FF85E05CFF4F20813181E054F0402F5FDF
:105E70003F4F2F733070DF01AE5BBF4F8D919C9110
:105E8000119728173907D1F3E05CFF4F808191818A
:105E9000E054F040E80FF91F6083EE85FF85E05C79
:105EA000FF4F31832083EE89FF89208181E090E0DC
:105EB0000F8C02C0880F991F0A94E2F7282B2083C9
:105EC00081E089A3EC89FD8980818064808381E001
:105ED00090E0DF91CF9108958F929F92AF92BF9201
:105EE000CF92DF92EF92FF920F931F9300D000D0DA
:105EF0000F92EDB7FEB7319684E0ADB7BEB71196FD
:105F00008C9383E0818387E0828385E0838381E0D3
:105F1000848389E396E061EB75E045EF55E025EC7D
:105F200030E004EC10E0B0ECEB2EF12CA1ECCA2E2A
:105F3000D12CF2ECAF2EB12CE6EC8E2E912C0E94DF
:105F4000FF2D0F900F900F900F900F901F910F91BA
:105F5000FF90EF90DF90CF90BF90AF909F908F9089
:105F60000895CF93DF930E946F2A0E942428CAECE1
:105F7000DEE20E941C122097E1F30E94CA2EF9CFA4
:105F8000629FD001739FF001829FE00DF11D649F1D
:105F9000E00DF11D929FF00D839FF00D749FF00DA9
:105FA000659FF00D9927729FB00DE11DF91F639F4A
:105FB000B00DE11DF91FBD01CF011124089597FB1C
:105FC000092E07260AD077FD04D086D006D00020FF
:105FD0001AF4709561957F4F0895F6F79095819525
:105FE0009F4F0895A1E21A2EAA1BBB1BFD010DC0F5
:105FF000AA1FBB1FEE1FFF1FA217B307E407F50779
:1060000020F0A21BB30BE40BF50B661F771F881F54
:10601000991F1A9469F760957095809590959B01EA
:10602000AC01BD01CF01089597FB092E05260ED0C6
:1060300057FD04D0D7DF0AD0001C38F450954095A6
:10604000309521953F4F4F4F5F4F0895F6F790954C
:106050008095709561957F4F8F4F9F4F08952F9238
:106060003F924F925F926F927F928F929F92AF92E8
:10607000BF92CF92DF92EF92FF920F931F93CF9335
:10608000DF93CDB7DEB7CA1BDB0B0FB6F894DEBFCC
:106090000FBECDBF09942A88398848885F846E84F2
:1060A0007D848C849B84AA84B984C884DF80EE803C
:1060B000FD800C811B81AA81B981CE0FD11D0FB645
:1060C000F894DEBF0FBECDBFED010895EE0FFF1FA8
:1060D0000590F491E02D0994AA1BBB1B51E107C068
:1060E000AA1FBB1FA617B70710F0A61BB70B881F68
:1060F000991F5A95A9F780959095BC01CD010895F7
:10610000911106C0803219F089508550D0F708955A
:0A611000992788270895F894FFCF1F
:10611A004E6F005965730054582074696D656F7528
:10612A007421006D6F64756C65206C6F636B6564B8
:10613A003F00486F70206368616E6E656C200020B6
:10614A0040200053004E2F4100386368002C002C79
:10615A00205B005D20280029004E4F5420454E4107
:10616A00424C45440053656E64696E6720736574DA
:10617A0074696E677320746F2052580A00526573EF
:10618A00657474696E672073657474696E677320C9
:10619A006F6E2052580A0041626F727465642065FE
:1061AA00646974730A00696E76616C696420736548
:1061BA006C656374696F6E000D0A496E76616C696D
:1061CA006420696E707574202D206469736361722E
:1061DA006465642107007363616E6E6572206D6F7A
:1061EA0064650053657474696E67732073617665BC
:1061FA006420746F20454550524F4D0A005265760F
:10620A0065727465642073657474696E6773206659
:10621A00726F6D20454550524F4D0A004C6F6164B4
:10622A00656420666163746F72792064656661755E
:10623A006C74730A004B657920616E64206368612F
:10624A006E6E656C732072616E646F6D697A6564D7
:10625A000A004F70656E4C52536E67205458207373
:10626A0074617274696E672000206F6E204857202F
:10627A000050504D00525353490053444100534378
:10628A004C00525844005458440041494E004C4274
:10629A004545500053504B54524D005342555300FC
:1062AA0053554D44004C4C494E440000342B3400A5
:1062BA003800382B340031320031322B3400313679
:1062CA000001000000C01200001A400AA1204EA5D9
:1062DA00001B1E27522C23308025000005400AA1EE
:1062EA00204EA50020244EA52C2330004B0000068A
:1062FA00400AD0009D49007B289D492C233000E1AB
:10630A00000005400A4501D7DC03B81E0EBF002372
:10631A002E48E801008A400A6001555502AD1E2048
:10632A00000023C88025000005400AA1204EA500D0
:10633A0020244EA52C233000020002000200020095
:10634A000200020002000200020002000200020033
:10635A0002000200020002FF01610265026A026E87
:10636A0002720276027A027E0284028B02900295FF
:10637A00029B029B029B029B0235019C02A002A285
:10638A0002A602A902AE02350100070B0C10111574
:10639A0000160A13223129000000002C2F9B2BB96A
:0863AA002EF32ED32E1C2F0050
:107E00000F92CDB7DEB7112484B714BE81FFF1D035
:107E100082E08093C00088E18093C10086E0809377
:107E2000C20080E18093C4008EE0CDD088249924E4
:107E3000CC24C394F5E0DF2EE1E1EE2E73E0F72EC3
:107E4000B6D0082F813479F4B2D08983C2D0898129
:107E5000823811F481E005C0813811F485E001C059
:107E600083E09ED09AC0823411F484E103C085344B
:107E700019F485E0B6D091C0853561F498D0082F0B
:107E800010E095D090E0982E8824802A912A880CC2
:107E9000991C82C0863521F484E0A3D080E0E1CF34
:107EA000843609F04CC083D082D0A82E80D0B82E62
:107EB00000E011E07CD0F80181938F01AE16D1F77C
:107EC00088D0FB2DF53489F4E0E0F1E00BC0F9999E
:107ED000FECF92BC81BC0894811C911C819180BD15
:107EE000FA9AF99AEA1598F358C08B2D863409F05E
:107EF00054C0F401F7BEE89507B600FCFDCFF401CD
:107F0000A0E0B1E02C9130E011968C91119790E0B7
:107F1000982F8827822B932B12960C01C7BEE895C9
:107F20001124329681E0A038B80761F7F401D7BE7A
:107F3000E89507B600FCFDCFE7BEE8952EC0843774
:107F4000F1F435D034D0182F32D0B82E42D0FB2DDA
:107F5000F63421F4F40105914F010CC0FB2DF534EA
:107F600049F4F999FECF92BC81BC0894811C911C04
:107F7000F89A00B5802F14D0115049F70EC08537FC
:107F800039F427D08EE10CD085E90AD08FE069CF93
:107F9000813511F488E017D01CD080E101D050CF9A
:107FA0009091C00095FFFCCF8093C600089580910A
:107FB000C00087FFFCCF8091C00084FD01C0A89560
:107FC0008091C6000895E0E6F0E098E19083808318
:107FD0000895EDDF803219F088E0F5DFFFCF84E10E
:107FE000DFCF1F93182FE3DF1150E9F7F2DF1F9166
:0E7FF0000895282E80E0E7DFEE27FF27099492
:027FFE0001057B
:0400000300007E007B
:00000001FF
